:10000000A6C0DAC0BFC0BEC0BDC0BCC051C2BAC06D
:10001000B9C0B8C0B7C0AECED9CEB4C0B3C0B2C0FC
:10002000B1C0B0C0AFC03DC43CC43BC4BFC4BEC47B
:10003000BDC4BCC4BBC4BAC471C473C496C4A9C48F
:10004000ABC4B2C45BC763C765C76BC779C75DC7BD
:1000500079C77AC77FC7A3C7A2C78CC78DC79EC7FA
:100060000600FF0901A101150026FF0075088501A2
:10007000953F0900B28001850495070900B280010F
:100080008505950F0900B28001850695100900B21B
:10009000A0018503953F0900B200018502953F0943
:1000A00000B200018507953F0900B20001C00403BA
:1000B00009045A0355006E00690063006F006E006A
:1000C000740072006F006C006C00650072007300B9
:1000D000200068007400740070003A002F002F00A8
:1000E0007700770077002E0075006E0069006300CE
:1000F0006F006E00740072006F006C006C00650091
:10010000720073002E0063006F006D000E03550037
:100110004E0043003000780078001201100100000A
:100120000008C016DF054000010203010902220099
:1001300001010080F0090400000103000000092112
:1001400001010001224E000705810308006411240B
:100150001FBECFE5D4E0DEBFCDBF10E0A0E6B0E02B
:10016000EAE7FFE102C005900D92A83BB107D9F77D
:1001700013E0A8EBB0E001C01D92A437B107E1F78E
:10018000A8D1F9CE3DCFA82FB92F80E090E041E073
:1001900050EA609530E009C02D91822797958795A8
:1001A00010F084279527305EC8F36F5FA8F3089599
:1001B000EADF8D939D930895CF93CFB7CF93C395E7
:1001C000839BE9F7839B09C0839B07C0839B05C082
:1001D000839B03C0839B01C0A3C0DF93C0915703DF
:1001E000DD27C25ADC4F839B02C0DF91EBCF2F93F8
:1001F0000F931F9300B32FEF03FB20F94F933F930F
:1002000010B34FEF012703FB21F93BE031C04E7FD4
:10021000012F10B3216028C0102F4D7F22600000F5
:1002200000B329C04B7F2460012F000010B32BC006
:1002300010B3477F28602AC04F7E00B320612CC0D6
:100240004F7D10B320622FC04F7B00B3206432C0BB
:10025000422700B349934FEF0000102713FB20F90A
:1002600010B31C70C9F1297F91F2012703FB21F91A
:1002700000B3237F89F2315058F1102713FB22F984
:1002800010B3277E79F2012703FB23F92F7C81F23B
:1002900000B3102713FB24F92F7971F200C010B3BB
:1002A000012703FB25F92F7359F200C000B3102773
:1002B00013FB26F9223040F200C010B3012703FBE4
:1002C00027F9243028F64F77206810B30000F9CFC3
:1002D00010E41ABF002719C03B503195C31BD04012
:1002E00010E41ABF0881033CF9F00B34E9F02091C7
:1002F00055031981110F1213EDCF4A81441F09369E
:1003000041F10D3211F0013E29F700935C033F915A
:100310004F911F910F912F91DF91CAB7C6FD4FCF1B
:10032000CF91CFBFCF91189520915C03222379F311
:1003300010915A03112369F534306AF130935A034E
:1003400020935603109157033BE0311B3093570322
:1003500022C000915A030130E4F40AE54F7049F4D9
:100360003091B60034FD19C00093B600CEE3D3E05F
:1003700018C03091490334FD10C000934903CAE40A
:10038000D3E00FC02795A8F45150A9F4220F000024
:10039000F9CF4AE503C042ED01C0432FC4E1D0E0EC
:1003A00032E011B31C60939A11BB02B320E41CE04D
:1003B0005F93012756E002BB279520F4515021F4AA
:1003C000220FF9CF012756E000003B5A02BBD0F2C2
:1003D000279528F4515029F4220F0000F9CF012766
:1003E00056E0279502BB20F4515021F4220FF9CF9B
:1003F000012756E02991332302BB21F6037F109198
:100400005B03110FC651D04002BB11F0109355038E
:1004100010E41ABF086011B3137F402F437F5F9130
:1004200000C000C002BB11BB42BB71CFEF92FF9274
:100430001F93CF93DF93FC018381833091F58281F9
:10044000833079F535E0E32EF12CC70176DD182FE6
:10045000F701E258FF4FE081CE2FD0E082958F70F8
:100460005AD7CC0FDD1FFE01E05AFF4F90E0918379
:100470008083812F8F704FD7CE59DF4F90E09983C3
:1004800088830894E108F1088FEFE8168FEFF806EB
:10049000E1F680E690E090935903809358038EE153
:1004A00001C080E0DF91CF911F91FF90EF90089500
:1004B0001F920F920FB60F9211248F931DBC1CBC7C
:1004C00081E08093B8008F910F900FBE0F901F9026
:1004D0001895A4D10DD7A5D688E10FB6F89481BDA3
:1004E00011BC0FBEE3DA8B9A20E048EB5BE003C05F
:1004F000CA010197F1F72150D9F78B9806D8789463
:1005000025D41092B80085B7806885BF889585B7D7
:100510008F7785BFD8DAA4D664D58091B8008823B8
:1005200081F38091540290915502A0915602B091AE
:1005300057020196A11DB11D80935402909355025C
:10054000A0935602B0935702DBD6CCD234D27ED8D9
:100550002AD5D7CF9091CC02882311F092959F7025
:10056000892F8F7008951F9381E0F4DF882311F4A1
:1005700010EF41C026B386B346B366B390E08095D2
:10058000909588709070F3E096958795FA95E1F7CD
:10059000E5E0880F991FEA95E1F730E02095309566
:1005A000227030703695279554E0220F331F5A95EC
:1005B000E1F7182F122B50E0409550954071507084
:1005C00034E0569547953A95E1F726E0440F551FDC
:1005D0002A95E1F7142B70E0609570956072707049
:1005E00095E0769567959A95E1F77695762F66274B
:1005F00077956795162B80E0ADDF882311F48FE0A7
:1006000003C083B380958F70812B1F910895E82FCD
:1006100082958F708C3069F48E2F8F708A30E0F461
:10062000E82FF0E0EE0FFF1FE85DFC4F8FEF8083B7
:100630000895A8E2B3E09FEFEF3F41F08C918E3038
:1006400031F411968C9111978E1709F49C931296A0
:1006500083E0AC33B80781F7089590915B02E92FEE
:10066000F0E0E45CFD4F80A39F5F9F7190935B027D
:1006700080915A02981721F49F5F9F7190935A02BC
:10068000089510925A0210925B0208950F931F93DF
:1006900080E060DF843011F010E001C01FE081E0F5
:1006A00059DF843011F000E001C000EF012B42B3AC
:1006B00022B382B362B330E02072307075E03595BA
:1006C00027957A95E1F7220F331F90E080749070A0
:1006D00036E0959587953A95E1F7880F991F880F31
:1006E000991F282B50E040715070B4E05595479504
:1006F000BA95E1F7242B661F6627661F660F660F03
:10070000660F622B609350021091B90010232BDF0B
:10071000082B0095102B109351021F910F910895F3
:100720001F93CF93DF93BC01CFEDD2E0A0E4B2E002
:10073000FC0140E050E011E088818077803719F0BB
:1007400020E030E00EC020E08091B90090E0042E5F
:1007500002C0959587950A94E2F780FF21E0212752
:1007600030E06115710529F08D919C91119791836D
:1007700080832D933D934F5F5F4F24963296483090
:100780005105D1F6DF91CF911F91089580E090E05F
:10079000C7DF10925002E7DE80935102109253029D
:1007A000109252026EDFDFDE8093B9008FEF2FCF01
:1007B0000F931F93882359F4A8E2B3E0E0E08C91F3
:1007C0008F3F49F0EF5F1296EA30C9F724C0E82F57
:1007D000E051EA3000F5AE2FB0E06F3039F4AA0FE7
:1007E000BB1FA85DBC4F8FEF8C9315C0FD01EE0FB2
:1007F000FF1FE85DFC4F6083AA0FBB1FFD01E450A3
:10080000FD4F45A7AA0FBB1FA050BD4F0D931D93D1
:100810002D933C9313971F910F9108958CEC92E0C8
:1008200060E170E040E350E078DB80E093DE8F3001
:1008300021F48FE284BB15BA04C080E284BB8FE050
:1008400085BB81E087DE843031F487B3857C87BB4C
:1008500088B38A6305C087B38A6387BB88B3857C06
:1008600088BB81B3806F81BB82B38F7082BB82E013
:100870008EBD8091CE029091CF029BBD8ABD89B77B
:10088000806189BF83CF0F931F93CF93DF93162F80
:10089000E82FF0E0EF30F10508F088C0ED5EFF4F83
:1008A000099490E0EC01CC0FDD1FCC0FDD1FC45785
:1008B000DF4F20E030E0462F50E0DC01AA0FBB1FE5
:1008C000A856BF4F1881CA01022E02C09595879580
:1008D0000A94E2F7837090708230910559F083306A
:1008E000910579F0019799F4ED91FC911197808130
:1008F000812B0CC0ED91FC91119780811095812383
:1009000005C0ED91FC91119780818127808321960C
:100910002E5F3F4F28303105A9F648C0862F02D6FA
:1009200045C0462F50E04F705070169516951C70BC
:100930008FE090E0012E02C0880F991F0A94E2F721
:1009400080959095209152023091530282239323F7
:10095000012E02C0440F551F0A94E2F7842B952BF9
:10096000909353028093520221C0C0E0D0E0062F42
:1009700010E0C8010C2E02C0959587950A94E2F705
:1009800080FF02C08C2F47D02196C830D10589F74F
:100990000DC0862F3CDE0AC084E890E055D4812F3C
:1009A00047D48AE05ADE02C0862F15D1DF91CF915D
:1009B0001F910F910895FF920F931F93CF93DF9391
:1009C000C8E2D3E08E0108521040FF24FA94288137
:1009D0002F3FA1F0F80180819181A281B38101971D
:1009E000A109B10980839183A283B3830097A105F4
:1009F000B10521F4F882822F698145DF22960C5FD0
:100A00001F4FF3E0CC33DF0711F7DF91CF911F9138
:100A10000F91FF900895EF92FF920F931F93CF9342
:100A2000DF93E82EC82FD0E081E090E00E2C02C0CA
:100A3000880F991F0A94E2F7F090B900F822FE019E
:100A4000EE0FFF1FEE0FFF1FE454FD4F82A18F70CA
:100A5000E0E0F0E0FF2011F4E1E0F0E08E01000FB3
:100A6000111F000F111F04541D4FE00FF11F60A153
:100A70000ADFF80183A1282F30E0FF2019F480E479
:100A800090E002C080E290E082239323892B51F012
:100A9000FE01EE0FFF1FE05CFD4F8081918101960A
:100AA00091838083FF2019F488E090E002C084E005
:100AB00090E082239323892B71F0FF2011F48DE2C3
:100AC00001C08BE280938800F0E3EF0EE092890092
:100AD00087E890E0B9D3DF91CF911F910F91FF90FC
:100AE000EF900895EF92FF920F931F93CF93DF93B0
:100AF0003ADD1091B900182780E02CDD843011F028
:100B000004E001C000E0C12FD0E081E0E82EF12C2C
:100B1000043020F081E01EDD843051F5202F30E0DC
:100B2000CE01002E02C0959587950A94E2F7F9014F
:100B3000E554FF4F80FF15C080818150808388235A
:100B4000A1F4C701002E02C0880F991F0A94E2F792
:100B50009C018091B90082278093B900802F5BDFD0
:100B600004C08091D0028F5F80830F5F083080F2D5
:100B7000DF91CF911F910F91FF90EF900895FF9219
:100B80000F931F93CF93DF93F82EEB016B816623B6
:100B900021F48981688177DE18C0EA81F0E0E37092
:100BA000F070EE0FFF1FEE0FFF1FE256FF4F70E0D9
:100BB00080E090E0208131814281538176D98B01A0
:100BC0009C018F2D69814881F3DDDF91CF911F91C9
:100BD0000F91FF900895CF92DF92EF92FF920F93C3
:100BE0001F93DF93CF93CDB7DEB728970FB6F89456
:100BF000DEBF0FBECDBF682F8091BA00873008F0EE
:100C000096C0603308F093C070E0E3E0660F771F92
:100C1000EA95E1F760587F4F8E010F5F1F4FC801C3
:100C200048E050E07AD98091BA008F5F8093BA0093
:100C30004885242F30E0C901807F9070803E910567
:100C4000C1F56EE0E62EF12C6801EE2D8E2D63E0ED
:100C50004BD9492F923011F400E010E0E595FF27C1
:100C6000E7FDF095EC0DFD1D8081E0FC03C020E068
:100C700030E002C024E030E090E002C09595879516
:100C80002A95E2F78F70907054E0000F111F5A956B
:100C9000E1F7082B192B442319F4812F602FF3DD82
:100CA0000894E108F1088FEFE8168FEFF80669F66F
:100CB00039C0403F31F0403FA8F1445F443090F5E7
:100CC00007C08E816D81DFDD8F81B80158DF2AC0BA
:100CD00023703070220F331F220F331F8091520276
:100CE0009091530202C0969587952A95E2F78F70EE
:100CF000282F30E04F81842F82958F7090E08217EB
:100D000093071CF08E816D810CC0842F90E08F7052
:100D10009070821793071CF08C816B8102C08A81CE
:100D20006981B1DD8091BA0081508093BA00289624
:100D30000FB6F894DEBF0FBECDBFCF91DF911F91EC
:100D40000F91FF90EF90DF90CF9008959091D30294
:100D50009F73892F8150803328F4903309F490E0F9
:100D6000892F39CF08958CEC92E060E170E040E388
:100D700050E0EBC8CF93DF93CCEDD2E0CE0162EB35
:100D800070E0E6D2249682E0CC3FD807B9F7CE01D6
:100D90008C976EEA70E0DCD2F9DCDF91CF91089598
:100DA000853011F088E001C080E18093050185EC79
:100DB00090E090933D0380933C0308950F931F931D
:100DC000282F85EC90E02093C500233061F024307B
:100DD00020F4223009F04BC00CC02630F9F0273047
:100DE00009F045C022C01092C30050DC8CE392E0B1
:100DF00010C01092C40086ED9FE2AFE3B0E0809394
:100E0000C0029093C102A093C202B093C3028CEBC4
:100E100092E090933D0380933C0341C090933D0347
:100E200080933C0301967CDC3AC08091C300882308
:100E300079F480E880937D0221E020937E028CE7A4
:100E400092E090933D0380933C032093C30027C01E
:100E500081E08093FD0282E08093FE028CEF92E0BD
:100E600090933D0380933C031092C30018C005EC9F
:100E700010E06091C40070E086E0660F771F8A95ED
:100E8000E1F7C80140E450E048D88091C4008F5F8A
:100E900087708093C40010933D0300933C0380E46B
:100EA0001F910F9108950F931F932091050126170D
:100EB00008F4622FDC0190E00BC08D91E0913C03BF
:100EC000F0913D038193F0933D03E0933C039F5FDA
:100ED000961798F3822F861B80930501882311F0C3
:100EE00080E05EC08091C60090E0FC017597EE3016
:100EF000F10508F054C0EE5DFF4F099489EC90E0D5
:100F000060E170E044E050E020D888DC48C080ED2B
:100F100092E012C089EC90E064E070E042E050E0C2
:100F20003BC08091C70090E087709070880F991F38
:100F3000880F991F84529D4F69EC70E009D22FC031
:100F400012DF2DC017DF2BC08091CA006091C9004D
:100F50009ADC25C00091CD001091CE002091CF00E9
:100F60003091D0008091C9006091C8004091C700C5
:100F70001FDC15C086DB13C06091C700603378F4B6
:100F800070E093E0660F771F9A95E1F760587F4F06
:100F900088EC90E048E050E0D8D701C0B6D281E0BC
:100FA0001F910F91089580910601883019F4AD9832
:100FB0001092060180910601873031F46CD78823A6
:100FC00019F088E08093060108951F93182F8295E9
:100FD0008F70A1D14FD7812F8F709DD14BD71F918B
:100FE00008955F926F927F928F929F92AF92BF927D
:100FF000CF92DF92EF92FF920F931F93DF93CF93E5
:101000000F92CDB7DEB713E0612EB4E05B2EACE0FB
:10101000AA2EA1E0BA2EF2E0EF2EE9E0FE2E75E056
:10102000972E6E010894C11CD11C66E0762E57E005
:10103000852EDFC0122F822F78D1582F1D3009F452
:10104000D8C01A30A1F580910601853069F57092FB
:101050000601AD9A8AE30ED780910801B6DF809130
:101060000701B3DF00E011C0E0913C03F0913D03C4
:10107000E20FF31F1081812FA8DF812F82958F70DF
:1010800081278F7048D1F6D60F5F202F30E08091F6
:101090000D01992787FD9095281739072CF38AE0D1
:1010A000E9D680920601A5C010920601A2C01A33AB
:1010B00041F481E08093060110920801109207012B
:1010C00045C080910601882309F493C05F3F09F46D
:1010D00062C08230F1F1833020F4813009F089C0A0
:1010E00006C08330E9F1843009F083C041C0852F08
:1010F000992787FD9095209107013091080144E0E0
:10110000220F331F4A95E1F7822B932B909308010E
:101110008093070180910B018F5F80930B018430D6
:1011200009F067C089E091E064E070E042E050E0DF
:10113000F4D6209107013091080180910901909126
:101140000A012817390739F5E092060110920B01C0
:1011500050C05295507F50930C016092060149C0D7
:1011600080910C01852B80930C015092060141C0A7
:1011700040910C01842F90E08F709070242F229565
:101180002F7030E082279327252F332727FD3095B6
:101190008217930719F0F09206012BC080910B0182
:1011A0008F5F80930B01815081F44983842F845099
:1011B000823030F4842FF4DDC60161E074DE17C0A4
:1011C000842FFCDD80930D010FC08CE091E061E085
:1011D0006ADE882361F081E080930D01B0923D03C7
:1011E000A0923C0310920C019092060102C0E09282
:1011F000060127D69C0180709B71892B09F41ACFB8
:101200000F90CF91DF911F910F91FF90EF90DF90A2
:10121000CF90BF90AF909F908F907F906F905F9096
:1012200008958091CD02882309F486E290E0F2C50A
:101230001F93182F82958F706ED00FDA812F8F70C9
:101240006AD00BDA1F910895CF93DF93EC0102C0AF
:10125000219603DA88818823D9F7DF91CF91089509
:101260001F938091D10280FF20C020915B0290915A
:101270005A022917D1F08091490384FF16C09217B2
:1012800010F4622F01C060E2691B162F693008F06C
:1012900018E0892F90E0845A9D4F612F4AD58091A4
:1012A0005A02180F1F7110935A021F910895FC01E2
:1012B000808180768032B9F48181813071F48281BD
:1012C0007DDD282F882369F080913C0390913D03B8
:1012D000909359038093580307C0893021F4828189
:1012E0005FDD2FEF01C020E0822F0895DCCD08954F
:1012F000C29ABA9A0895C29887E080930E01089521
:10130000C29908C080910E01815080930E018823FC
:1013100009F4C29A08958A3010F4805D08958031EE
:1013200010F08FE30895895C0895982F80538A30D8
:1013300070F0892F8156863010F4865F0895892FCA
:101340008154863010F08FEF0895892F87530895C8
:10135000DC01FB01838113968C9313978281129693
:101360008C931297818111968C93119780818C9325
:101370000895C09AB89A0895C098B89A80EA95E0FE
:101380000197F1F7B898C09A80EC90E00197F1F7D7
:1013900086B3E0EEF4E03197F1F7B09902C081E056
:1013A0000895817008951F93182FC098B89A88E007
:1013B0008A95F1F7112311F0B898C09A84E38A95C1
:1013C000F1F7B09B10E08CEA8A95F1F7C09AB898D3
:1013D0006111CFDF88E28A95F1F7812F1F9108957F
:1013E000817060E0E0CF0F931F93182F08E0812FEA
:1013F0008170F6DF1695811110680150C1F7812FB9
:101400001F910F9108950F931F93182F08E0812FBC
:101410008170013011F060E001C061E0C4DF169519
:1014200081111068015099F7812F1F910F91089534
:101430008FEFD9CFDF92EF92FF920F931F93CF934D
:10144000DF93E82EEB0198DF882381F580EFCBDF77
:1014500080E4FF24182F98EFD92ED80E81E0C0DF4A
:10146000082F81E0BDDF882329F0002371F08EEF83
:10147000F82E1EC0002349F41E1528F0888180FF35
:1014800004C0E11611F0F12E01E0802FA9DF888160
:1014900086958883002311F08068888311501D157C
:1014A000E9F6112329F02196812FD4CFFF24FA9455
:1014B0008F2DDF91CF911F910F91FF90EF90DF90D3
:1014C0000895FF920F931F93CF93DF93082FEB01A3
:1014D000F42E52DF209741F085E585DF18E08991F1
:1014E00082DF1150E1F702C08CEC7DDFFF2019F0A4
:1014F000802F89DF02C0802F76DFDF91CF911F918F
:101500000F91FF90089540E0DCCF10928C02109272
:10151000940210929C021092A4021092AC021092BB
:10152000B4020895CF92DF92EF92FF920F931F9330
:10153000DF93CF93CDB7DEB728970FB6F894DEBF11
:101540000FBECDBF682F669566959CEFE92EE82A01
:10155000603340F570E083E0660F771F8A95E1F70E
:1015600060587F4FCE01019648E050E0D6D4CE01BE
:10157000019667E08BD2888700E06E010894C11C59
:10158000D11CFE2CF0948AE5B601BDDF8E2D2BDF39
:101590008F2D29DF4DDF182F4BDFEEDE015011F0CC
:1015A0001A3A89F728960FB6F894DEBF0FBECDBF62
:1015B000CF91DF911F910F91FF90EF90DF90CF902F
:1015C0000895EF92FF920F931F93CF93DF9390E0D4
:1015D00033E0880F991F3A95E1F7EC01C058DF4FCF
:1015E0008B0127E8E22EF12CE80EF91ECE01A5D4DE
:1015F000F8019081891711F080E007C021960F5FF4
:101600001F4FCE15DF0591F781E0DF91CF911F913C
:101610000F91FF90EF9008951F93CF93DF93182FB2
:10162000EA018091D202862369F087E516D8812FDE
:1016300014D817E08F81FCDD115021971F3FD1F79F
:101640008AE00BD8DF91CF911F9108953F924F927E
:101650005F926F927F928F929F92AF92BF92CF9242
:10166000DF92EF92FF920F931F93DF93CF93CDB74B
:10167000DEB76B970FB6F894DEBF0FBECDBF80917B
:10168000D20287FFD9C1809115018F5F8F7080933F
:101690001501882309F07DC06FDE882309F079C029
:1016A000CC24CA944E010894811C911C89E0A82E78
:1016B000B12CAC0EBD1E8C2DB401BCDEC82E8E5FCD
:1016C000823008F4B9C14CE852E06FEF20E030E01E
:1016D000D22EFA0180818823A1F0D401F90103E020
:1016E000EE0FFF1F0A95E1F7E457FD4F9C918081B3
:1016F000981731F411963196AA15BB05B9F73DC07C
:10170000D62E2F5F3F4F485F5F4F2630310509F4DB
:101710008EC16D2DDDCF8BE260E4A4017DDFD401AD
:10172000ED2DFF27E7FDF09513E0EE0FFF1F1A9553
:10173000E1F7E457FD4F8D918193AA15BB05D9F7C9
:101740008091D20283FF19C0EE2407E810E0C8019F
:10175000F4D3F82EFFE2F81740F08E2DB40131DFFC
:10176000882319F08EE06F2D8ED8F7FC06C0E39425
:10177000085F1F4F20E3E21651F7ED2DFF27E7FD2D
:10178000F095E15FFE4F809154028083CC2009F0F8
:1017900092CF3090D20280E138225090D1029FE067
:1017A000592AEFE2E51510F070E3572E66E0A62EF9
:1017B000CE014A969B8F8A8FAA94EA2CFF24870138
:1017C00053E0000F111F5A95E1F704571D4FF80120
:1017D0002081222309F427C1F701E15FFE4F909198
:1017E00054028081981B591638F48DE260E2A801FA
:1017F00013DFF801108217C1332009F414C19D30A2
:1018000008F011C1283231F02A3309F4BDC020316B
:1018100009F009C180911501833061F46A2D70E0EF
:1018200043E0660F771F4A95E1F764577D4F84E4E4
:101830006ADEF9C08B3009F0F6C08A2C992433E0B7
:10184000880C991C3A95E1F78CE892E0880E991E75
:101850008EEBB40158DE8E010F5E1F4FE9DDF801FB
:1018600081938F018A8D9B8DE817F907B9F7CE0117
:10187000419668E00BD1998D891709F0D4C08A8907
:1018800090E0D82ECC24898990E0C82AD92AF70183
:1018900083E0EE0FFF1F8A95E1F7E457FD4F80814B
:1018A000803129F403E0CC0CDD1C0A95E1F7F70147
:1018B000EE0FFF1FE058FD4F6080718090E06916C9
:1018C00090E8790639F080E090E0E0E46E16E5E01B
:1018D0007E0614F081E090E0482E8091D20282FFD3
:1018E00049C0BB2407E810E0C80127D38037C9F5F9
:1018F0008B2DB40166DE8823B1F16B2D70E0B3E06F
:10190000660F771FBA95E1F768577F4FCE010996AA
:1019100048E050E002D388898E3761F5442029F4ED
:101920008B859C858615970554F48B859C858C1535
:101930009D051CF08F856E850EC0442029F4898595
:101940009A856816790644F489859A85C816D90659
:101950001CF08F856D8597D7B394FEE2FB1568F672
:1019600009C087FD07C0B394085F1F4F2FE2B2166E
:1019700009F0BACFEE0CFF1C80E892E0E80EF91EE9
:10198000F701D182C0824FC080911501873009F0E4
:101990004AC08701F3E0000F111FFA95E1F70457E1
:1019A0001D4FE7E0DE2E85EFB801ADDD41DDC82E2D
:1019B000DA94FFEF8F1711F4DD20A9F78C2D90E05A
:1019C0008C010095109574E0159507957A95E1F7CF
:1019D000082719270F70107023C02ADDC81681F45C
:1019E0000115110569F4EE0CFF1CF701E058FD4FDD
:1019F000C0828CE792E0E80EF91EF701158212C052
:101A0000FFEFCF1661F4EE0CFF1C80E892E0E80EC9
:101A1000F91E8FEF9FEFF7019183808303C0DA9463
:101A2000DD20D9F6A9DCAA2009F0C6CE05C09FEFBB
:101A3000D91609F070CEAACE6B960FB6F894DEBF19
:101A40000FBECDBFCF91DF911F910F91FF90EF900F
:101A5000DF90CF90BF90AF909F908F907F906F90CE
:101A60005F904F903F900895982F28E048E1862F8F
:101A70008927382F317080FD942796953111906811
:101A8000215011F06695F3CF892F08951F93CF93BE
:101A9000DF93EC01162F80E003C06991E5DF115060
:101AA0001123D9F7DF91CF911F91089585B78260F7
:101AB00085BF8BB780648BBF8BE480934A038AE534
:101AC0008093490308951F93CF93DF9310915A0396
:101AD000135017FDD3C080915703CCE0D0E0C81B52
:101AE000D109C25ADC4F07DC809156038D3209F0D0
:101AF000B2C0183009F0C0C083EC80933E038AE581
:101B00008093B600109216018881807621F0CE0174
:101B1000CEDB282F8DC09A811092470389818823BC
:101B200021F41092480322E07CC0853019F4909390
:101B30005B0376C0863009F05FC08B81813049F449
:101B40008AE191E0909359038093580380E422E165
:101B500050C0823049F48CE291E090935903809315
:101B6000580380E422E245C0833049F58A81882306
:101B700049F48EEA90E0909359038093580380E4EF
:101B800024E037C0813049F482EB90E09093590310
:101B90008093580380E42AE52CC0823049F48CE01D
:101BA00091E0909359038093580380E42EE021C084
:101BB0008330D9F4CE013AD4282F80E01AC0813284
:101BC00049F48EE391E0909359038093580380E4A5
:101BD00029E00FC0823249F480E690E090935903E7
:101BE0008093580380E42EE404C0CE011FD4282F34
:101BF00080E4809316011CC0883021F421E08DE53B
:101C000093E011C0893019F490935D0309C08A30C4
:101C100011F421E006C08B3019F48BE480934A0361
:101C200020E087E493E0909359038093580309C020
:101C30002F3F39F4888187FD2E8180E8809316013B
:101C400006C08F81882319F48E81821708F0822FB5
:101C50008093B70011C08091160187FF0DC0CE019F
:101C6000612F44DB8F3F21F48EE18093B60004C0E6
:101C7000882311F01092B70010925A038091B60099
:101C800084FF49C08091B7008F3F09F444C0182FEA
:101C9000893008F018E0811B8093B70080913E03E3
:101CA00098E8892780933E03112341F1209158033E
:101CB000309159038091160186FF0DC0AFE3B3E068
:101CC00080E090E0F901E80FF91FE491ED930196AF
:101CD0001817C1F708C0D901912FEFE3F3E08D91F8
:101CE00081939150E1F71150812F90E01F5F019691
:101CF000820F931F90935903809358038FE393E0CF
:101D0000612F56D2612F6C5F6C3019F08FEF80938A
:101D1000B7006093B60094E180B38C7031F49150B9
:101D2000D9F710925B0310925503DF91CF911F9169
:101D300008951F93DC01162F8091490384FF07C08B
:101D400080914A0398E8892780934A0303C08AE573
:101D500080934903912FEBE4F3E08D9181939150AF
:101D6000E1F78BE493E0612F23D21C5F10934903CA
:101D70001F9108951F920F920FB60F9211242F9367
:101D80008F939F93EF93FF939BB12CB1E091390216
:101D9000EF5FEF7180913A02E81711F492E007C00B
:101DA0009871E0933902F0E0E95EFD4F2083809165
:101DB0003B02982B90933B02FF91EF919F918F9163
:101DC0002F910F900FBE0F901F9018951F920F929A
:101DD0000FB60F9211248F939F93EF93FF939091DF
:101DE000370280913802981759F0E0913802EF5F7E
:101DF000E0933802F0E0E95EFE4F80818CB901C0CB
:101E00005598FF91EF919F918F910F900FBE0F907A
:101E10001F9018959C011092370210923802109270
:101E2000390210923A0297FF03C082E08BB93F77E4
:101E3000832F992780BD29B988E98AB986E880BDB2
:101E400008959091390280913A02981719F480E030
:101E500091E00895E0913A02EF5FEF71E0933A026A
:101E6000F0E0E95EFD4F808190913B0210923B02D1
:101E700090E00895282F909137029F5F809138025B
:101E80009817E1F3E92FF0E0E95EFE4F208390938D
:101E90003702559A0895909137028091380220E0D8
:101EA000981709F421E0822F0895629FD001739F53
:101EB000F001829FE00DF11D649FE00DF11D929FE6
:101EC000F00D839FF00D749FF00D659FF00D992725
:101ED000729FB00DE11DF91F639FB00DE11DF91F49
:101EE000BD01CF011124089587FB082E062687FD2A
:101EF000819567FD619505D00EF4919507FC81955C
:101F00000895991B79E004C0991F961708F0961B55
:101F1000881F7A95C9F780950895DC01CB01FC01F3
:101F2000E199FECF06C0FFBBEEBBE09A31960DB241
:101F30000D9241505040B8F70895E199FECF9FBBF4
:101F40008EBBE09A99278DB30895DC01CB0102C0C6
:101F50002D9105D041505040D8F70895262FE19992
:101F6000FECF9FBB8EBB2DBB0FB6F894E29AE19AD1
:0A1F70000FBE01960895F894FFCF0C
:101F7A001E0330003000300030003A0030003000DC
:101F8A00300030003A0030003000300030000301E9
:101F9A0008060D0B413A004C2B300A0010204080F5
:101FAA00020810200102040832003800350001003E
:101FBA0000006400000070170000407E0500020067
:081FCA000000000000705AFF46
:00000001FF
